:100000000C9463000C948B000C948B000C948B006C
:100010000C948B000C948B000C948B000C948B0034
:100020000C948B000C948B000C948B000C948B0024
:100030000C948B000C948B000C948B000C948B0014
:100040000C943F020C948B000C94C1030C948B0015
:100050000C948B000C948B000C948B000C948B00F4
:100060000C948B000C948B000000000024002700EF
:100070002A0000000000250028002B0000000000DE
:1000800023002600290004040404040404040202DA
:100090000202020203030303030301020408102007
:1000A0004080010204081020010204081020000012
:1000B0000007000201000003040600000000000029
:1000C00000008D000A0511241FBECFEFD4E0DEBF73
:1000D000CDBF11E0A0E0B1E0E8E0FEE002C0059095
:1000E0000D92A032B107D9F711E0A0E2B1E001C052
:1000F0001D92AE3CB107E1F710E0C6ECD0E004C0C1
:100100002297FE010E94FE06C23CD107C9F70E9459
:1001100038020C9402070C94000080910C0190911D
:100120000D0190932B0180932A010895EF92FF9285
:100130000F931F9382E10E947203892B09F04BC039
:1001400091E090932901809128018823C9F590932B
:10015000280110922D0110922C011AC0A9016627C6
:1001600057FD6095762F8BEB91E020E030E00E9408
:10017000640664E170E080E090E00E94A10280915A
:100180002C0190912D01019690932D0180932C01CB
:1001900080912C0190912D0120910A0130910B0149
:1001A0000597E4F280910C0190910D0190932B0141
:1001B00080932A012E5F3F4F30930B0120930A0159
:1001C0000E94930260932001709321018093220189
:1001D000909323015AC083E10E947203892B09F096
:1001E00052C080912901882371F40E949302609388
:1001F000240170932501809326019093270181E0CB
:100200008093290142C00E949302209124013091E1
:1002100025014091260150912701621B730B840B2D
:10022000950B605177428040904078F110922D01FB
:1002300010922C0119C08BEB91E040E050E060E09F
:1002400070E020E030E00E94640664E170E080E04D
:1002500090E00E94A10280912C0190912D010196C5
:1002600090932D0180932C0180912C0190912D0170
:1002700005970CF31092280181E090E090930B0118
:1002800080930A0102C010922901809128018130D7
:1002900009F0BEC00E9493027B018C018091200175
:1002A00090912101A0912201B0912301E81AF90A4D
:1002B0000A0B1B0B60912A0170912B01882777FD97
:1002C0008095982F21E934EF40E050E00E947906B4
:1002D000E616F7060807190708F49AC00E94930269
:1002E0006093200170932101809322019093230158
:1002F00010922D0110922C011FC040910A015091C3
:100300000B0141505040662757FD6095762F8BEBCF
:1003100091E020E030E00E94640664E170E080E05B
:1003200090E00E94A10280912C0190912D010196F4
:1003300090932D0180932C0180912C0190912D019F
:100340000597DCF210922D0110922C0124C02B3065
:10035000310544F4A901662757FD6095762F8BEB94
:1003600091E006C08BEB91E040E050E060E070E08F
:1003700020E030E00E94640664E170E080E090E0FC
:100380000E94A10280912C0190912D0101969093E1
:100390002D0180932C0180912C0190912D012091B1
:1003A0000A0130910B01059794F22330310529F4AD
:1003B00080910E0190910F0117C02530310529F46D
:1003C00080911001909111010FC02730310529F45F
:1003D000809112019091130107C02930310541F439
:1003E000809114019091150190932B0180932A0123
:1003F000C901029690930B0180930A010D9741F475
:1004000081E090E090930B0180930A011092280103
:100410001F910F91FF90EF9008950F931F930BEB97
:1004200011E0C80140E05BE460E070E00E94FE0380
:10043000C80160E071E00E949A0582E160E00E94DC
:10044000050383E160E00E9405038DE061E00E9406
:10045000050382E161E00E94250383E161E00E94DF
:1004600025038DE061E00E9425031F910F910895FF
:100470000E94CB020E940D020E949600FDCF1F92A7
:100480000F920FB60F9211242F933F934F935F93C8
:100490006F937F938F939F93AF93BF93209132017C
:1004A0003091330140913401509135017091360102
:1004B000DA01C9010296A11DB11D672F6A5F6D3770
:1004C00030F06D57DA01C9010396A11DB11D60938B
:1004D00036018093320190933301A0933401B0939D
:1004E000350180912E0190912F01A0913001B091A2
:1004F00031010196A11DB11D80932E0190932F0112
:10050000A0933001B0933101BF91AF919F918F9132
:100510007F916F915F914F913F912F910F900FBEFF
:100520000F901F9018958FB7F89420913201309159
:10053000330140913401509135018FBFB901CA0197
:100540000895EF92FF920F931F937B018C018FB759
:10055000F8944091320150913301609134017091CF
:1005600035018FBF2FB7F8948091320190913301FC
:10057000A0913401B09135012FBF841B950BA60BC0
:10058000B70BE816F9060A071B0760F71F910F91D2
:10059000FF90EF900895789484B5826084BD84B50F
:1005A000816084BD85B5826085BD85B5816085BD6E
:1005B000EEE6F0E0808181608083E1E8F0E0808118
:1005C00082608083808181608083E0E8F0E08081C8
:1005D00081608083E1EBF0E0808184608083E0EBE8
:1005E000F0E0808181608083EAE7F0E080818460D0
:1005F000808380818260808380818160808380812C
:10060000806880831092C1000895282F30E0C901CE
:1006100086569F4FFC0194912A573F4FF9018491D0
:10062000882391F0E82FF0E0EE0FFF1FE859FF4F0D
:10063000A591B491662329F48C91909589238C938C
:1006400008958C91892B8C930895482F50E0CA010E
:1006500082559F4FFC012491CA0186569F4FFC0191
:1006600094914A575F4FFA0134913323D1F12223F9
:1006700031F1233021F4809180008F7705C0243040
:1006800031F4809180008F7D8093800018C02130EC
:1006900019F484B58F7704C0223021F484B58F7D9E
:1006A00084BD0DC0263021F48091B0008F7705C045
:1006B000273029F48091B0008F7D8093B000E32F24
:1006C000F0E0EE0FFF1FEE58FF4FA591B4916623A7
:1006D00029F48C91909589238C9308958C91892B82
:1006E0008C930895682F70E0CB0182559F4FFC01D9
:1006F0002491CB0186569F4FFC0144916A577F4F4E
:10070000FB019491992319F420E030E038C02223B2
:1007100031F1233021F4809180008F7705C024309F
:1007200031F4809180008F7D8093800018C021304B
:1007300019F484B58F7704C0223021F484B58F7DFD
:1007400084BD0DC0263021F48091B0008F7705C0A4
:10075000273029F48091B0008F7D8093B000892FDD
:1007600090E0880F991F84589F4FFC01A591B49188
:100770008C9120E030E0842311F021E030E0C901C9
:1007800008951F920F920FB60F9211242F933F934B
:100790004F935F936F937F938F939F93AF93BF9389
:1007A000EF93FF934091C600E091B701F091B8013B
:1007B000CF01019660E870E00E9498069C0180914C
:1007C000B9019091BA012817390739F0E95CFE4F59
:1007D00040833093B8012093B701FF91EF91BF910F
:1007E000AF919F918F917F916F915F914F913F91C9
:1007F0002F910F900FBE0F901F9018955F926F92E0
:100800007F928F929F92AF92BF92CF92DF92EF92A0
:10081000FF920F931F93CF93DF93EC013A014B01AB
:10082000413281EA580787E0680780E078070CF0DA
:100830007FC060E472E48FE090E0A40193010E9425
:10084000CD062150304040405040CA01B90122E05D
:1008500030E040E050E00E94CD0659016A01A60157
:100860009501209530954095509594E0220F331FC7
:10087000441F551F9A95D1F760E072E18AE790E036
:100880000E94CD06CA01B9012FEF30E040E050E0F0
:100890000E947906A40193010E94CD06C9018150EE
:1008A0009F4F181619061CF4522E5A9403C0552453
:1008B0005394521A60E874E88EE190E0A401930129
:1008C0000E94CD062150304040405040CA01B9013D
:1008D00022E030E040E050E00E94CD0620953095C7
:1008E0004095509583E0220F331F441F551F8A9572
:1008F000D1F760E072E18AE790E00E94CD06CA017C
:10090000B9012FEF30E040E050E00E947906A401E9
:1009100093010E94CD06C90181509F4F18161906F8
:100920001CF4822F815002C081E0821B851500F5E6
:10093000E885F98581E090E00A8802C0880F991F58
:100940000A94E2F7808360E874E88EE190E0A40105
:1009500093010E94CD062150304040405040CA01D2
:10096000B90122E030E040E050E00E94CD0604C032
:10097000E885F98510829501EC81FD813083EE8157
:10098000FF812083EA85FB85208141E050E0CA0198
:100990000E8402C0880F991F0A94E2F7282B208347
:1009A000EA85FB852081CA010F8402C0880F991F48
:1009B0000A94E2F7282B2083EA85FB85808108884A
:1009C00002C0440F551F0A94E2F7842B8083DF9105
:1009D000CF911F910F91FF90EF90DF90CF90BF903C
:1009E000AF909F908F907F906F905F900895FC01E3
:1009F000A085B18521898C9190E0022E02C0959549
:100A000087950A94E2F780FFF6CF0484F585E02D00
:100A1000608308958AE191E09093BC018093BB01CB
:100A200087E391E09093BE018093BD0185EC90E057
:100A30009093C0018093BF0184EC90E09093C20139
:100A40008093C10180EC90E09093C4018093C30136
:100A500081EC90E09093C6018093C50186EC90E014
:100A60009093C8018093C70184E08093C90183E01B
:100A70008093CA0187E08093CB0185E08093CC010D
:100A800081E08093CD0108950F931F93CF93DF935F
:100A90008C01EB0109C02196D801ED91FC910190E8
:100AA000F081E02DC801099568816623A1F7DF91E7
:100AB000CF911F910F910895EF92FF920F931F9383
:100AC000CF93DF938C017B01EA010CC0D7016D91BC
:100AD0007D01D801ED91FC910190F081E02DC801DC
:100AE00009952197209791F7DF91CF911F910F9151
:100AF000FF90EF900895DC01ED91FC910280F3816D
:100B0000E02D099508950F931F938C01DC01ED9161
:100B1000FC910190F081E02D6DE00995D801ED91F7
:100B2000FC910190F081E02DC8016AE009951F91C8
:100B30000F9108950F931F938C010E947B05C801AC
:100B40000E9483051F910F9108952F923F924F921B
:100B50005F926F927F928F929F92AF92BF92CF924D
:100B6000DF92EF92FF920F931F93DF93CF93CDB756
:100B7000DEB7A0970FB6F894DEBF0FBECDBF1C0145
:100B80006A017B01411551056105710549F4DC01DC
:100B9000ED91FC910190F081E02D60E3099554C046
:100BA000882499245401422E55246624772401E098
:100BB00010E00C0F1D1F080D191DC701B601A30180
:100BC00092010E94AB06F80160830894811C911C7D
:100BD000A11CB11CC701B601A30192010E94AB0682
:100BE000C901DA016C017D01C114D104E104F104F1
:100BF000F1F681E0E82EF12CEC0EFD1EE80CF91C5C
:100C00003E010894611C711CD501C4010197A10922
:100C1000B1096C01C818D90814C0F601EE0DFF1D0A
:100C200060816A3010F4605D01C0695CD101ED91B2
:100C3000FC910190F081E02DC10109950894E10833
:100C4000F1086E147F0449F7A0960FB6F894DEBF42
:100C50000FBECDBFCF91DF911F910F91FF90EF900D
:100C6000DF90CF90BF90AF909F908F907F906F90CC
:100C70005F904F903F902F900895EF92FF920F93C7
:100C80001F93CF93DF93EC017A018B0177FF0FC0A5
:100C9000E881F9810190F081E02D6DE209951095D0
:100CA0000095F094E094E11CF11C011D111DCE0192
:100CB000B801A7012AE00E94A505DF91CF911F91FD
:100CC0000F91FF90EF900895DC012115310541F45B
:100CD000ED91FC910190F081E02D642F099508952C
:100CE0002A30310519F40E943D0608950E94A50599
:100CF0000895629FD001739FF001829FE00DF11D66
:100D0000649FE00DF11D929FF00D839FF00D749F85
:100D1000F00D659FF00D9927729FB00DE11DF91F31
:100D2000639FB00DE11DF91FBD01CF01112408958E
:100D300097FB092E07260AD077FD04D049D006D0AC
:100D400000201AF4709561957F4F0895F6F79095FD
:100D500081959F4F0895A1E21A2EAA1BBB1BFD018E
:100D60000DC0AA1FBB1FEE1FFF1FA217B307E4078A
:100D7000F50720F0A21BB30BE40BF50B661F771FE2
:100D8000881F991F1A9469F76095709580959095C2
:100D90009B01AC01BD01CF01089597FB092E0526EB
:100DA0000ED057FD04D0D7DF0AD0001C38F4509580
:100DB0004095309521953F4F4F4F5F4F0895F6F77F
:100DC00090958095709561957F4F8F4F9F4F0895B7
:100DD000AA1BBB1B51E107C0AA1FBB1FA617B70761
:100DE00010F0A61BB70B881F991F5A95A9F780957D
:100DF0009095BC01CD010895EE0FFF1F0590F49171
:080E0000E02D0994F894FFCFE6
:100E0800456D70657A616D6F730001000200050021
:100E18000A000500050000000000F70444055C0511
:00000001FF
